:020000040000FA
:06000000CA3001303A286D
:08000800A000030EA100831209
:1000100005191128831601178312B2308100B1012E
:100020002C2883160113831203140B190310A80D37
:10003000A90DAA0DAB0DAC0DAC16FF302C02031DA3
:100040002C28FA302B02031D2C2832152A08AF0069
:100050002908AE002808AD008B100B11210E83007B
:06006000A00E200E0900B5
:04006600003400342E
:0C007400203084008001840A80300402E7
:10008000031C3C28DA2183160C3085058701831276
:10009000850187010730990000309A0010308316DF
:1000A0008E008312603083168F0083120030831617
:1000B00091009F008312C830831681008312313073
:1000C0009000003083168C00831210308B00BD1B13
:1000D0006F2885196F286400851D6B28E722CE22C2
:1000E00081018E018F010B118B100B108C018B176E
:1000F000872032199320B40B852803108519031427
:10010000BA0DF0303A0203193C212D2378286400FF
:100110003310B10A311F9228AC01AB01AA01A90129
:10012000A801B101080032110130B7008B13203053
:10013000370783169B001C141A088312A400103082
:10014000370783169B001C141A088312A300A6000D
:100150000230A6060030370783169B001C141A08CD
:100160008312A200A7000130A7068B17331CBE28FC
:1001700022090339A200A309A409A50924082F0212
:10018000031D362923082E02031D362922082D02BD
:10019000031D362901303702031DD3283E18D3280A
:1001A0003E143F14FC2102303702031DDC28BE1828
:1001B000DC28BE143F140B2203303702031DE52850
:1001C0003E19E5283E153F14172204303702031D5F
:1001D000EE28BE19EE28BE153F1423220530370243
:1001E000031DF7283E1AF7283E163F143222063028
:1001F0003702031D0029BE1A0029BE163F144122F2
:1002000007303702031D09293E1B09293E173F14F9
:10021000502208303702031D1229BE1B1229BE17B7
:100220003F145B2209303702031D1B295E181B296E
:100230005E143F1466220A303702031D2429DE189B
:100240002429DE143F1471220B303702031D2D299F
:100250005E192D295E153F147C220C303702031DD8
:100260003629DE193629DE153F148722B70A0D30EC
:1002700037020318080096280130B600B400B50014
:10028000B70085018701B2138720B40B54290310EE
:1002900085190314BA0DF0303A0203197C29B50B05
:1002A00054299630B5008621321D44293211331C61
:1002B0005E292D090339AD00AE09AF092F1C442971
:1002C0002D083002031944292D08B0002E1E4429A0
:1002D0008B1320303707BC002F08BB00C52110301E
:1002E0003707BC002E08BB00C52100303707BC0013
:1002F0002D08BB00C5218B1785018701B70AB60100
:100300000D303702031C4429CE2208000130370289
:100310000319922202303702031997220330370261
:1003200003199C22043037020319A1220530370239
:100330000319A622063037020319AB220730370211
:100340000319B022083037020319B52209303702E9
:100350000319BA220A3037020319BF220B303702C1
:100360000319C4220C3037020319C92208003F1CAC
:1003700008003F101030BC003E08BB00C5213030E3
:10038000BC005E08BB00C52108008B133B08831628
:100390001C159A0083123C0883169B0055309D0063
:1003A000AA309D009C1464009C18D3291C11831250
:1003B0008B170800831600309B001C141A08831248
:1003C000BD00831610309B001C141A088312BE0057
:1003D000831630309B001C141A088312DE00FF3095
:1003E000C800CA15CB15CC15CD15CE15CF15D01517
:1003F000D115D215D3150800C130BE05FF30DE057A
:100400001130C405C0000030C200C600BD185F1422
:10041000BD18DF140800C230BE05FF30DE05023013
:10042000C405C0000030C200C6005F100800C43020
:10043000BE05FF30DE050630C405C0000030C20036
:10044000C6005F100800C830BE05FF30DE0518305A
:10045000C405C0000030C200C600BD185F14BD183E
:10046000DF140800D030BE05FF30DE053030C40593
:10047000C0000030C200C600BD185F14BD18DF14F4
:100480000800E030BE05FF30DE053030C405C00096
:100490002030C200C600BD185F14BD18DF1408006C
:1004A0007F30BE05C030DE05C030C505C10000305C
:1004B000C300C7000800BF30BE05C030DE053030C5
:1004C000C505C1000030C300C70008003F30BE05AD
:1004D000C130DE059030C505C1000030C300C70043
:1004E00008003F30BE05C230DE05C030C505C10082
:1004F0000030C300C70008003F30BE05C430DE0531
:10050000C030C505C1000030C300C70008003F303F
:10051000BE05C830DE05C030C505C1000030C300CF
:10052000C70008001030850602308706080020301A
:1005300085060030870608002130850600308706D2
:100540000800023085060230870608000030850664
:10055000063087060800003085060630870608004A
:1005600000308706183087060800003085062130E5
:10057000870608000030850609308706080000302D
:10058000870618308706080000308706183087066F
:100590000800003087061830870608003E18FC2146
:1005A000BE180B223E191722BE1923223E1A3222F0
:1005B000BE1A41223E1B5022BE1B5B225E186622E1
:1005C000DE1871225E197C22DE1987220800B6012E
:1005D000B401B5013D1CEF2ABD01BD14F12ABD01D6
:1005E0003D143D08B6006400F52AF62AF72AF82AD9
:1005F000F92AFF30B51B8500B51F8501B40BF32A1E
:10060000B50BF32A0310B60CB608031DF32A00300D
:10061000BC003D08BB00C521080005125C1805168A
:10062000DC1C8512DC1885165C1D05105C19051490
:10063000DC1D8510DC1985145C1E87105C1A87147C
:10064000DC1E0711DC1A07155C1F07105C1B071462
:10065000DC1F8712DC1B871608008F0803190800AF
:100660008F0178308E00C80F5F2DC80A441C5D2BA7
:10067000461C4E2BCA1C3F2BCA014A156B2B4A1D28
:10068000442BCA01CA156B2BCA1D492BCA014A1635
:100690006B2B4A1E6B2BCA01CA146B2B4A1D532BA2
:1006A000CA014A166B2BCA1D582BCA014A166B2B5E
:1006B0004A1E6B2BCA01CA146B2BCA1C622BCA01BF
:1006C0004A156B2B4A1D672BCA01CA156B2B4A1E94
:1006D0006B2BCA014A15C41C922BC61C832BCB1C46
:1006E000742BCB014B15A02B4B1D792BCB01CB15BC
:1006F000A02BCB1D7E2BCB014B16A02B4B1EA02B72
:10070000CB01CB14A02B4B1D882BCB014B16A02B60
:10071000CB1D8D2BCB014B16A02B4B1EA02BCB0141
:10072000CB14A02BCB1C972BCB014B15A02B4B1D17
:100730009C2BCB01CB15A02B4B1EA02BCB014B151B
:10074000441DC72B461DB82BCC1CA92BCC014C1526
:10075000D52B4C1DAE2BCC01CC15D52BCC1DB32BE2
:10076000CC014C16D52B4C1ED52BCC01CC14D52B43
:100770004C1DBD2BCC014C16D52BCC1DC22BCC0156
:100780004C16D52B4C1ED52BCC01CC14D52BCC1C08
:10079000CC2BCC014C15D52B4C1DD12BCC01CC1521
:1007A000D52B4C1ED52BCC014C15C41DFD2BC61DC5
:1007B000EE2BCD1CDF2BCD014D155F130B2C4D1DEA
:1007C000E42BCD01CD150B2CCD1DE92BCD014D1604
:1007D0000B2C4D1E0B2CCD01CD140B2C4D1DF32BD2
:1007E000CD014D160B2CCD1DF82BCD014D160B2C2C
:1007F0004D1E0B2CCD01CD140B2CCD1C022CCD018C
:100800004D150B2C4D1D072CCD01CD150B2C4D1E60
:100810000B2CCD014D155F1B342C441E342C461E71
:10082000252CCE1C162CCE014E15422C4E1D1B2CF9
:10083000CE01CE15422CCE1D202CCE014E16422CC0
:100840004E1E422CCE01CE14422C4E1D2A2CCE011F
:100850004E16422CCE1D2F2CCE014E16422C4E1E73
:10086000422CCE01CE14422CCE1C392CCE014E157A
:10087000422C4E1D3E2CCE01CE15422C4E1E422C3B
:10088000CE014E15C41E692CC61E5A2CCF1C4B2CF3
:10089000CF014F15772C4F1D502CCF01CF15772C42
:1008A000CF1D552CCF014F16772C4F1E772CCF0123
:1008B000CF14772C4F1D5F2CCF014F16772CCF1DF7
:1008C000642CCF014F16772C4F1E772CCF01CF14FD
:1008D000772CCF1C6E2CCF014F15772C4F1D732C0E
:1008E000CF01CF15772C4F1E772CCF014F15DF1876
:1008F000A02C451EA02C471E912CD01C822CD00170
:100900005015AE2C501D872CD001D015AE2CD01D0B
:100910008C2CD0015016AE2C501EAE2CD001D01411
:10092000AE2C501D962CD0015016AE2CD01D9B2CF9
:10093000D0015016AE2C501EAE2CD001D014AE2CCF
:10094000D01CA52CD0015015AE2C501DAA2CD001C6
:10095000D015AE2C501EAE2CD0015015DF18D72C60
:10096000C51ED72CC71EC82CD11CB92CD1015115BE
:10097000E52C511DBE2CD101D115E52CD11DC32C68
:10098000D1015116E52C511EE52CD101D114E52CD5
:10099000511DCD2CD1015116E52CD11DD22CD101E8
:1009A0005116E52C511EE52CD101D114E52CD11C9A
:1009B000DC2CD1015115E52C511DE12CD101D115B3
:1009C000E52C511EE52CD1015115DF180F2D451FC7
:1009D0000F2D471F002DD21CF12CD2015215DF1311
:1009E0001D2D521DF62CD201D2151D2DD21DFB2C12
:1009F000D20152161D2D521E1D2DD201D2141D2DB5
:100A0000521D052DD20152161D2DD21D0A2DD201C7
:100A100052161D2D521E1D2DD201D2141D2DD21C79
:100A2000142DD20152151D2D521D192DD201D21592
:100A30001D2D521E1D2DD2015215DF18482DDF1B12
:100A4000482DC51F482DC71F392DD31C2A2DD30172
:100A50005315562D531D2F2DD301D315562DD31DB0
:100A6000342DD3015316562D531E562DD301D314B6
:100A7000562D531D3E2DD3015316562DD31D432DF8
:100A8000D3015316562D531E562DD301D314562D74
:100A9000D31C4D2DD3015315562D531D522DD3016B
:100AA000D315562D531E562DD3015315B72140088B
:100AB000C4004108C5005F18DF145F1CDF10480840
:100AC000C9000C304A05031D05120C304B05031DEF
:100AD00085120C304C05031D05100C304D05031D0F
:100AE00085100C304E05031D87100C304F05031D7B
:100AF00007110C305005031D07100C305105031D64
:100B000087120C305205031D07120C305305031DCC
:100B1000871149080E020318B92D12304A05031D2A
:100B2000051612304B05031D851612304C05031DAA
:100B3000051412304D05031D851412304E05031D9A
:100B4000871412304F05031D071512305005031D81
:100B5000071412305105031D871612305205031D6C
:100B6000071612305305031D8715FF30480203197D
:100B700008008F08031D0800872049080E02031C87
:100B8000B92D18304A05031D051206304A05031D0C
:100B9000051618304B05031D851206304B05031D45
:100BA000851618304C05031D051006304C05031D35
:100BB000051418304D05031D851006304D05031D25
:100BC000851418304E05031D871006304E05031D91
:100BD000871418304F05031D071106304F05031DFC
:100BE000071518305005031D071006305005031D6A
:100BF000071418305105031D871206305105031DD7
:100C0000871618305205031D071206305205031DC2
:100C1000071618305305031D871106305305031DB1
:040C2000871508002C
:084000000200030006000900A4
:02400E00CC33B1
:10420000010078007A007C007E007B0079007F004E
:104210007D007A0078007E007C007D007F007900C0
:104220000200F200F600FA00FE00F200F600FA00CA
:10423000FE00F200F600FA00FE00F200F600FA00BE
:10424000FF00050005000500050009000900090040
:1042500009000D000D000D000D00110011001100EE
:104260000100FF00FF00FF00FF00FF00FF00FF0054
:10427000FF00FF00FF00FF00FF00FF00FF00FF0046
:10428000FF007B00FF00FF00FF00FF00FF00FF00BA
:10429000FF00FF00FF00FF00FF00FF00FF00FF0026
:1042A000FF00FE00FF00FF00FF00FF00FF00FF0017
:1042B000FF00FF00FF00FF00FF00FF00FF00FF0006
:1042C000FF001100FF00FF00FF00FF00FF00FF00E4
:1042D000FF00FF00FF00FF00FF00FF00FF00FF00E6
:1042E000FF00FF00FF00FF00FF00FF00FF00FF00D6
:1042F000FF00FF00FF00FF00FF00FF00FF00DD00E8
:00000001FF
